:020000040000FA
:02000000B62820
:08000800F000030EF1008B1A59
:100010000B1D0D283D200B1136280B1A8B1C1328A5
:1000200057208B103628831603130C1E1D288312AD
:1000300003130C1E1F285C2036288312031383161B
:1000400003138C1E2828831203138C1E2B2869206F
:100050008312031336280B1F3628831603138C1FB5
:100060003628831203138C1F36287F208312031334
:10007000710E8300F00E700E090075088100F219F0
:10008000442872194A280800BA100000061ABA1447
:100090003A1508007D08C100411C86120000411875
:1000A0008616C1144108FD00BC3081000800721999
:1000B0005A28F2150B120800200884000008990045
:1000C000A00ABE0B0800831603130C12831203133D
:1000D0000800F214450884001A0880006114C50A5B
:1000E000E003031961158C1E7928E114840A6C2839
:1000F0000800981C7D28181218160800080008002F
:100100001430E500E401E3010000E30B8428E40B74
:100110008328E50B822808000A30E500E401E301AA
:100120000000E30B9028E40B8F28E50B8E280800D5
:100130000230E500E401E3010000E30B9C28E40B3E
:100140009B28E50B9A280800EC308F0078308E0051
:10015000A928831603130C10831203130C1090109C
:1001600010140C1CB12810100C10080007309F0050
:10017000831603138A3081008312031381018316CF
:10018000031310308500133086008312031385019A
:10019000003086008615A4200617A42005118316BA
:1001A00003131812831203139817831603131815D9
:1001B0008130990083120313830120308400800171
:1001C000840A841FDF28A03084008001840A031D74
:1001D000E5288317203084008001840A841FEC28DE
:1001E00083132130A0004630C500A03083160313CE
:1001F000B000831203138515982085119820F20111
:10020000F2140130DF00F2150130FA0000308B00EB
:100210000B178B17F219132972192429F2182D299B
:10022000721839290A2901308A007A0882070C29B4
:10023000432962296C299B29A229DD29E029192A51
:100240009B2AC52AD12ADB2A01308A003D08820771
:100250000E294E2B5D2B722B9C2B01308A005F08E0
:1002600082071029CF2BDF2BF12BF92BFC2B0F2C26
:10027000232C01308A003F08820712292A2C462CA1
:100280005B2C702C8B2C72190C2986112130A0004C
:100290008D210530FA00F2118B10851598208511FB
:1002A00098200B160C293A1C5929061E55293A107C
:1002B0005D29061A59293A145D2908007A08F900BF
:1002C0000230FA003A1D0C293A117908FA000800A8
:1002D0007A08F9000330FA003A1D6C293A11BA1C69
:1002E000822981018B120B11061A74290B19862998
:1002F0000108693C031C8829A03081000F3081026D
:100300008B1608000A308A290B308A290C308A297A
:100310000D308A29F400F21708007A08F9008316D4
:1003200003130C10831203130C109010EC308F0089
:1003300078308E0010140C1C9B2910100C107908BA
:10034000FA0008008D218D218D213230F700E83030
:100350008F0090308E0010149D308100AB30F5007E
:100360000B118B163A1DB2293A11F7033A14BA1839
:100370003A103A1DB9293A113A18C2290000BA1C9C
:10038000CD29C429BA18CD2900000C1CB929F217AF
:100390000430F4007708F400192B0130BA06F70B8B
:1003A000C4298B1210100C100730FA00E02910102D
:1003B0008B120B110C30FA000C290730FA000C29B3
:1003C0000C1010108F016C30F5008E006430F700B7
:1003D000061AE829061EEA2910140F1CED29061A30
:1003E000F829101075088E000F10F70BEA29092A5A
:1003F0000F10A1308E000F1CFB29061A022A0830AC
:10040000FA00192A1010F2170130F4000C30FA002B
:100410000C291010F2170230F4000C30FA000C29ED
:10042000F2130009F700840A00087702031D3B1449
:100430000800BA01F701F717213084000F10BC3013
:100440008E0010140F1C222A1010061ABA143A1526
:10045000AB30F5006821F21B962A0830F800FC0149
:100460003A1D302A3A110310BA1C382A0314FC0A28
:10047000800C840AFC0E3A1D3B2A3A110310BA1C68
:10048000432A0314FC0A800C8403FC0EF80B302A68
:10049000BA113A123A1D4A2A3A11BA18BA153A1D37
:1004A0004F2A3A11BA183A161130FC05F801BA1958
:1004B00078143A1A78167808FC06BB103B117C18A1
:1004C000BB147C1A3B15F2130009C200840A000811
:1004D00084034202031D3B143B123B1C752ABB1CC8
:1004E000752ABB188A2A3B16752A3B1E7B2A840A6A
:1004F0000009840380000008F71BF700840AF70B4B
:100500002A2A8B120B128615061705118D210A3027
:10051000FA000C29F2170330F400982AF21707307A
:10052000F400982AF2170830F400982AF400982A68
:100530000C30FA000C29BA01F70121308400053093
:100540008000840AE301E4010530E3000830E400A0
:10055000AB30F50081000B118B160830E4003A1D1A
:10056000AF2A3A110310BA180314800CE40BAF2A17
:10057000840AE30BAD2A8B1221308400FA01F211B8
:10058000BA0172140130BF000C29831603130C103A
:100590008312031390108F018E0110140B30FA0098
:1005A0000C290F1FD12A1010FA01F211BA0172148E
:1005B0000130BF000C298B120B128615061705158A
:1005C0008D212008840007308000840A4530800097
:1005D000840A52308000840A52308000840A20301D
:1005E0008000840AF701F8017408C200F70A0A3093
:1005F000C2020318F62AC207F703303077078000DB
:10060000840AF701F70A0130C2020318022BF7032C
:100610003030770780008515982085119820851542
:1006200098208511FA01F211F21372140130BF0003
:100630000C298B120B128615061705158D21200823
:10064000840007308000840A54308000840A5230CD
:100650008000840A41308000840A20308000840AAF
:10066000F701F8017408C200F70A0A30C202031841
:10067000342BC207F703303077078000840AF70174
:10068000F70A0130C2020318402BF7033030770716
:1006900080000B2B3D08F9000130BD00FD1C4E2BE6
:1006A000FD107D19592B000000000130FD067D155D
:1006B0004E2B7D117908BD0008008615A420A420CA
:1006C0000613A4200511BC3081000B118B167D3060
:1006D000BC007D104A23BC0B692B7D144A230330D8
:1006E000BD00722B4630C50084000008C4000830ED
:1006F000BC00C3017D144A23450884000008C200E1
:100700007D10421C862B00007D14C30A4A23C20CB4
:10071000BC0B802B7D10431C8E2B7D144A23C40BF5
:100720009A2B8B1290108F018E0110140430BD0093
:100730000E299C2BC50A772B8F1D9C2B1010BD01F9
:1007400072110617A420A420051585158C2085118B
:100750000130DF00F2140E294630C5008400000885
:10076000C4000830BC00450884000008C2007D10A9
:10077000FD10421CBD2B00007D14FD1CBD2BFD1087
:10078000C20CBC0BB72BC40BCD2B8B1290108F015E
:100790008E0110140430BD000E29C50AB12B46305D
:1007A000C500FF30E0008C12831603138C1618135B
:1007B0008312031318160230DF00F2101029611C97
:1007C000F02B463084000008E000E00317306002A0
:1007D000031CEC2B0230E000E11800000330DF00C6
:1007E0001029611DF12B4630C5000630DF000F2CAB
:1007F00010290630DF0010291730BE002130A0007C
:100800004630C500450884000008E2002008840046
:1008100062088000A00AC50ABE0B022C0F2CF21938
:1008200010290B12F210DF01E101831603138C1261
:1008300083120313851598208511982018127215BC
:100840000230BD001029F2107214DF01E101013005
:10085000BF0010298B120B128316031306150C16FA
:100860001815813099001812181383120313981762
:100870002130A000200884000008BE000230BF0024
:100880008316031398168312031312293E08031DBF
:10089000122983160313981C582C981283120313E1
:1008A000BF0172102130A0000130FA00F2151229A8
:1008B00083120313122927308400800A3A30000281
:1008C000031C6D2C303080008403800A3A30000213
:1008D000031C6D2C30308000840A0530BF001229C3
:1008E0002130A0002008840017308000840A4E3098
:1008F0008000840A42308000840A3A308000840AF2
:1009000020308000840A30308000840A303080003B
:100910000130BF0012299630BE00831603130C105D
:10092000831203130C1090108F018E0110140C1CF5
:10093000972C10100C10BE0F942C0130BF00122900
:02400E00223F4F
:00000001FF
